:0200000480007A
:100000006F004005732F2034930F8000630AFF03B5
:10001000930F90006306FF03930FB0006302FF038A
:10002000170F0000130F0F2B63040F0067000F0062
:10003000732F203463540F006F00400093E19153FD
:10004000171F000023203FFC171F0000232E0FFA6C
:100050006FF01FFF930000001301000093010000E8
:10006000130200009302000013030000930300003A
:100070001304000093040000130500009305000022
:10008000130600009306000013070000930700000A
:1000900013080000930800001309000093090000F2
:1000A000130A0000930A0000130B0000930B0000DA
:1000B000130C0000930C0000130D0000930D0000C2
:1000C000130E0000930E0000130F0000930F0000AA
:1000D000732540F16310050097020000938202012E
:1000E000739052307350447497020000938202015F
:1000F00073905230735000189702000093820202EE
:1001000073905230B70200809382F2FF7390023BEB
:100110009302F0017390023A73504030970200004E
:1001200093824201739052307350203073503030BC
:100130009301000097020000938202ED7390523009
:10014000130510001315F501634C05000F00F00FA7
:10015000930110009308D005130500007300000000
:1001600093020000638A020073905210B7B200003D
:100170009382921073902230735000303725000024
:100180001305058073200530970200009382420119
:1001900073901234732540F17300203093012000D6
:1001A000733000C093030000631C700E9301300095
:1001B000732000C0930300006314700E930140008D
:1001C000737000C093030000631C700C9301500017
:1001D000736000C0930300006314700C930160000F
:1001E000733020C093030000631C700A93017000F9
:1001F000732020C0930300006314700A93018000F1
:10020000737020C093030000631C7008930190007A
:10021000736020C093030000631470089301C00052
:10022000733000C893030000631C70069301D00074
:10023000732000C893030000631470069301E0006C
:10024000737000C893030000631C70049301F000F6
:10025000736000C8930300006314700493010001ED
:10026000733020C893030000631C700293011001D7
:10027000732020C8930300006314700293012001CF
:10028000737020C893030000631C70009301300159
:10029000736020C893030000631470006310300281
:1002A0000F00F00F638001009391110093E11100A2
:1002B0009308D00513850100730000000F00F00FB4
:1002C000930110009308D00513050000730000008F
:1002D0006FF01FFD731000C0000000000000000060
:1002E000000000000000000000000000000000000E
:1002F00000000000000000000000000000000000FE
:1010000000000000000000000000000000000000E0
:1010100000000000000000000000000000000000D0
:1010200000000000000000000000000000000000C0
:1010300000000000000000000000000000000000B0
:081040000000000000000000A8
:040000058000000077
:00000001FF
